:03000000120003E8
:0300330002005276
:101932001993199719B919D719ED19FF1A091A1319
:03194200000000A2
:10000300E4F5D0C2AF75818F12001675D0001213BC
:03001300C780FEA5
:0C00160090193278087E197F45121929D4
:0100220022BB
:1019450012010101FF0000401D0700102F000102D8
:10195500030109023C00010104802B090400000673
:10196500FF000005070501024000010705020240CE
:10197500000107050302400001070581024000013F
:1019850007058202400001070583024000010403A8
:10199500090422034500690063006F006E00200002
:1019A50054006500630068006E006F006C006F00F6
:1019B500670079001E034500690063006F006E0033
:1019C5002000440049005600410020005500530006
:1019D500420016033C002D002D00530065007200E7
:1019E50023002D002D003E001203530074006100FA
:1019F5006E0064006100720064000A034900500033
:101A0500410043000A03300030003400370004036E
:101A15003F00020DF9020E7D020DFF020E14020EAB
:101A25002B020E36020E3F020E4D020E59020E66B5
:101A3500020E6F020E768000000000000200018198
:101A450000000000000200028200000065000200A4
:101A550003020300006500000005020100006500A7
:101A65000000078006000100007878088006000263
:101A7500000078780980067303787878780A8008FA
:101A85000000000001000B00096E00000000000CC2
:101A9500810A0000000001000D40E06E006C680046
:101AA500000F40E100006C6800001001180B0315E1
:101AB5005902159D0515AF0716090816420916574F
:101AC5000A166C0B17440C17530D17650E17740F78
:051AD50017861017AA9E
:0E002300ED1D6009EF0FF97700ED1D70F7225B
:100036007C05EC600D7DC6ED60041DED70FC1CECCE
:1000460070F31FBFFF011EEE4F70E522C0D053D8DC
:10005600EFD0D032907FA5E054406008907FA5E0B5
:10006600544070F8907FA57480F022907FA574406C
:10007600F022907FA6EFF0907FA5E05401700890E3
:100086007FA5E0540160F822907FA5E05401700836
:10009600907FA5E0540160F8907FA6E0228E1B8F2A
:1000A6001C8D1D12005A7FA2120078AF1B12007819
:1000B600AF1C120078AF1D12007812007112005AA0
:1000C6007FA2120078120071907FA5E0540260EDC5
:1000D600228E1E8F1F12005A7FA2120078AF1E12A8
:1000E6000078AF1F12007812007112005A7FA31217
:1000F6000078907FA57420F012008E12008EF520F5
:10010600120071E52022901B3EEFF0901B3FEDF0B0
:10011600907FE3741BF0907FE4743EF0907F98E04C
:1001260054EFF0907FE5E0907F98E04410F0907FE8
:10013600E5E022901B3EEFF0907FE3741BF0907F8A
:10014600E4743EF0907F98E054EFF0907FE5E0FF96
:10015600907F98E04410F0907FE5EFF0901B3FE031
:10016600228F21852118E521F45407C40354F8FD94
:100176007FC512010C907F98E04402F07404551874
:100186006007907F98E054FDF0228F228D23E523AF
:10019600600EAA2274010A1333C3DAFC4218800DDA
:1001A600AA2274010A1333C3DAFCF45218AF1812E8
:1001B6000167228F828E83E0FAEF2401F582E43E06
:1001C600F583E0C39A228F828E83E0FA04F0EF244F
:1001D60002F9E43EF8E92AF582E438F583E0228F55
:1001E600828E83E02DFAEF2402F9E43EF8E92AF53F
:1001F60082E438F583E022EF2401F582E43EF583BC
:10020600E08F828E83FAE0C39A1422AB05EF2401B5
:10021600F582E43EF583E0FA04F0EF2402F9E43EC9
:10022600F8E92AF582E438F583EBF0228F828E8393
:10023600E02DF0228F2A8D2B8B2C7F437E251201F9
:10024600FD24AD50667D027F437E251202117DFF9F
:100256007F437E25120211902649E0FD7F437E25CD
:100266001202117D077F437E25120211AD8C7F435A
:100276007E25120211AD2A7F437E25120211AD2B77
:100286007F437E25120211AD2C7F437E251202117B
:10029600AD277F437E25120211AD287F437E2512AE
:1002A6000211AD297F437E25120211902649E004F2
:1002B600F0228F2D8D2E7480652D60187421452DAA
:1002C600FF1201395404600C7421452DFF120139C7
:1002D600540470F4AD2E7421452DFF12010C2290AA
:1002E6007FE0E4F0907FE1F0907FDE740FF0907F86
:1002F600DFF0798F7701798FE725E0FA24C5F5825B
:10030600E4347FF583AA83AB827440F0E725E0FCF2
:1003160024B4F582E4347FF5837402F08B828A83F9
:100326007440F0E725E0FA24B4F582E4347FF583DF
:100336007402F007E724FC50BD7700798FE7FD7C57
:10034600007F077E011218FF74202FF53074203EBF
:10035600F52F853082852F83E4F0E5302401F58280
:10036600E4352FF583E4F0E5302402F582E52F34F9
:1003760001F583E4F0A3F0E5302404F582E52F349B
:1003860001F583E4F0E5302406F582E52F3401F526
:1003960083E4F0E5302405F582E52F3401F5837416
:1003A60010F007E724FA5093227D207FC912010C32
:1003B6007F0A7E001200367D007FC912010C7D1077
:1003C6007FCA12010C7D387FC412010C7DC77FC421
:1003D60012010C7D2F7F2012010C7D2F7F601201F0
:1003E6000C7D2A7FA012010C7DD57FC112010C2243
:1003F6008D318B327FB0120139F533E53114600649
:1004060014603A020479E532600B14601514601D1D
:10041600146022805E74EB55334408FD7FB01201F0
:100426000C22740C4533FD7FB012010C227D2B7F0C
:10043600B112010C227D037FB112010C22E532605C
:100446000B14601514601D146022802774EE55335A
:100456004402FD7FB012010C2274034533FD7FB0C8
:1004660012010C227D2B7FB112010C227D037FB17C
:1004760012010C228F34798977007D477FB11201F2
:100486000C7DCB7FA212010C7DB27FCC12010CE554
:100496003460077D0F7FB012010C228F35E53524BD
:1004A600FFB3E43324FFB3E433FA75F005A42476EE
:1004B600F9770075F005EAA42477F975F005EAA442
:1004C6002478F975F005EAA42479F975F005EAA40B
:1004D600247AF97D82742F4535FF12010C7D8074D4
:1004E600224535FF12010C7D30742C4535FF120173
:1004F6000C7D0774324535FF12010C7D07743345B8
:1005060035FF12010C228F368D37E53660267D03C6
:100516007FB112010C7D017FA112010C7987E76082
:1005260004798D7701798877007985E4F709F77979
:10053600897700227986E537F719E4F722AC387413
:10054600806F6033EF24FFB3E43324FFB3E433FA60
:1005560075F005A42476F9770175F005EAA42479E7
:10056600F9A70575F005EAA42478F9A70375F0053F
:10057600EAA4247AF9A704228F398D3A7480653962
:10058600700302069AE53924FFB3E43324FFB3E48B
:100596003375F005A42477F97701E53924FFB3E430
:1005A6003324FFB3E43375F005A42479F9E7FD7429
:1005B600324539FF12010CE53924FFB3E43324FF39
:1005C600B3E43375F005A42479F9E7FD74334539AE
:1005D600FF12010CE53924FFB3E43324FFB3E433FF
:1005E60075F005A42478F9E7600C7DE0742245399E
:1005F600FF12010C800A7D8074224539FF12010C1E
:10060600E53A60167D2F74304539FF12010C7D2FB7
:1006160074314539FF12010C80147D03743045395D
:10062600FF12010C7D0374314539FF12010CE539C7
:1006360024FFB3E43324FFB3E43375F005A4247830
:10064600F9E7602AE53924FFB3E43324FFB3E43342
:1006560075F005A4247AF9E7603A742C4539FF123F
:1006660001394480FD742C4539FF12010C22742295
:100676004539FF1201394408FD74224539FF12013C
:100686000C742F4539FF1201394408FD742F453982
:10069600FF12010C228F3B7480653B700302072515
:1006A600E53B24FFB3E43324FFB3E43375F005A43C
:1006B6002477F97700742F453BFF12013954F7FD73
:1006C600742F453BFF12010CE53B24FFB3E43324B2
:1006D600FFB3E43375F005A42478F9E76029E53B18
:1006E60024FFB3E43324FFB3E43375F005A4247A7E
:1006F600F9E76013742C453BFF120139547FFD74F2
:100706002C453BFF12010C7D01AF3B1202B87D4028
:10071600AF3B1202B87D807422453BFF12010C22CA
:100726008F3C7480653C6020E53C24FFB3E43324B1
:10073600FFB3E43375F005A42477F9E760031206E6
:100746009B7D01AF3C1202B8227FB1120139F53D03
:100756005402700302086879898729743C553D0361
:1007660003543FF528853D277B637D697F6312022D
:100776003A743C553D70030207FE24FC600F24F4D6
:10078600605024F0602E24F0600D02084A7D437FFD
:10079600B112010C0208647D637FB112010C7989E4
:1007A6007707798A77FF0977FF79887700798C77D9
:1007B600040208647989E7FA64076004EAB4080762
:1007C6007989770602086479887706798C77020238
:1007D60008647989E7FA64066004EAB4070B798944
:1007E6007708798C77010208647988E7B406028075
:1007F60003020864770880667D037FB112010C79D5
:1008060089E724F960051460068011798C770179EF
:100816008A77000977287987770080427989770077
:100826007985E7094760377988E760327D017FA1DE
:1008360012010C798D7701798A77FF0977FF79881C
:100846007700801A79898729743C553D0303543F04
:10085600F528853D277B317D4C7F3F12023A798E04
:100866007701228F3E8C3F8D408A418B42E53E24A4
:10087600FFB3E43324FFB3E43375F005A42478F919
:10088600874E754C40E53E23235403F54DE542243F
:1008960005F582E5413401F583E0F549E53EB4808E
:1008A600028003020921754E00754C20798EE7609F
:1008B6005AAF42AE411201FD24F3504FAD4DAF4247
:1008C600AE411202117D0CAF42AE41120211E54259
:1008D6002406F582E5413401F583E0FD04F0AF42DC
:1008E600AE411202117D09AF42AE411202117545A9
:1008F60000E5452485F9E7FDAF42AE411202110538
:1009060045E54524F750EA798E7700740455496029
:100916000AE524600612074F5349FBE5402404F517
:1009260082E53F3401F583E070237420453EFF12D3
:100936000139FA4549F54954106012E5402404F599
:1009460082E53F3401F583E54CF05349EFE5402459
:1009560004F582E53F3401F583E07003020EE1857C
:100966004082853F83E0FAE5402401F582E4353F85
:10097600F583E0C39AF54324FC4003020EE17D03B0
:10098600AF40AE3F1201E5FB7A00EB2404FBE43AEC
:10099600FAAD437C00D3EB9DEA9C30D202B2E7204D
:1009A600E703020EE1854082853F83E0FA04F0E525
:1009B600402402FDE4353FFCED2AF582E43CF58354
:1009C600E0F54D854082853F83E0FA04F0E540245A
:1009D60002FDE4353FFCED2AF582E43CF583E0F5C3
:1009E6004A854082853F83E0FA04F0E5402402FD13
:1009F600E4353FFCED2AF582E43CF583E0F54B85D2
:100A06004082853F83E0FA04F0E5402402FDE435A8
:100A16003FFCED2AF582E43CF583E0F544E540240D
:100A260006F582E53F3401F583E0FA654B602DE576
:100A3600402406F582E53F3401F583E0F529854B30
:100A460028853E277B557D4E7F4512023AE5402498
:100A560006F582E53F3401F583E54BF0E5402406D3
:100A6600F582E53F3401F583E004F0E54A603A1487
:100A7600602724FE600D14603014601D24FE6003A0
:100A8600020D8DAF3E120726E5402404F582E53FB0
:100A96003401F583E4F0020E8FE5402404F582E587
:100AA6003F3401F583E04480F0E5402404F582E517
:100AB6003F3401F583E0B4FF4FAD44AF40AE3F1283
:100AC60002327401654A600AE54AB40502800302EF
:100AD6000E8FE5402404F582E53F3401F583E0F509
:100AE60029854428853E277B627D617F5812023A1C
:100AF600E5402404F582E53F3401F583E4F07D0109
:100B0600AF3E1202B8020E8FE53EB480397FB112B5
:100B16000139543CFA6430602D7FB1120139C0E0CE
:100B2600AF40AE3F1201B9F52979898728D0028AEC
:100B3600277B317D447F2112023AAD44AF40AE3F60
:100B4600120232020E8FE5402404F582E53F34019D
:100B5600F583E0547FF545E544C395455003854448
:100B660045854082853F83E0F54FE5402402F553F5
:100B7600E4353FF552E5456014E553254FF582E42B
:100B86003552F583E0FDAF3E12010C054FC3E54536
:100B96009401F543602AE553254FF582E43552F575
:100BA60083E0F551054F901B3EF0907FE3741BF0F8
:100BB600907FE4743EF0907FE5E01543E54370D600
:100BC600854082853F83E54FF0E544C39545F5446E
:100BD600E5402404F582E53F3401F583E0C39545FD
:100BE600F0E5447003020C85854082853F83E0145E
:100BF600F0FCE5402402FBE4353FFAEB2CF582E4F9
:100C06003AF583E544F0854082853F83E014F0FCA5
:100C1600E5402402FBE4353FFAEB2CF582E43AF595
:100C260083E54BF0854082853F83E014F0FCE54088
:100C36002402FBE4353FFAEB2CF582E43AF583E532
:100C46004AF0854082853F83E014F0FCE5402402AB
:100C5600FBE4353FFAEB2CF582E43AF583E54DF0FB
:100C6600E5402404F582E53F3401F583E0547FF046
:100C7600E5402406F582E53F3401F583E54BF07443
:100C860024453EFF120139F54354C07003020D1985
:100C9600744055436024AF40AE3F1201B9F528E5D4
:100CA600422404F582E5413401F583E0F529853EC9
:100CB600277B527D557F5812023A74805543602433
:100CC600AF40AE3F1201B9F528E5422404F582E5AE
:100CD600413401F583E0F529853E277B527D4D7F22
:100CE6005812023AE54E7012E5402404F582E53FBB
:100CF6003401F58374FFF0020E8F7D01AF3E1202C0
:100D0600B8E5402404F582E53F3401F583E54CF06F
:100D1600020E8FE5402404F582E53F3401F583E0B9
:100D26006011E5402404F582E53F3401F583E05483
:100D3600806030754308E54E7014E5402404F58262
:100D4600E53F3401F583E05480600375430AAD4303
:100D5600AF3E1202B8E5402404F582E53F3401F5C2
:100D660083E4F07421453EFF12013954807003027A
:100D76000E8F752900752800853E277B4F7D587F8D
:100D86003F12023A020E8F754800754700754600FD
:100D9600E544600B1544AF40AE3F1201CCF546E585
:100DA60044600B1544AF40AE3F1201CCF547E54415
:100DB600600B1544AF40AE3F1201CCF548E54460E8
:100DC6000D1544AF40AE3F1201CCE54470F3854BA0
:100DD60029854A28853E277B657D787F6512023AFC
:100DE600E54A24F6B40C004003020E7D901A17FA69
:100DF6002A2A73752400020E8F7D637FB112010CBF
:100E0600798A770109779079877701020E8FE54015
:100E16002404F582E53F3401F583E4F07D017FA1EA
:100E260012010C8064AB48AD47AF461203F68059F9
:100E3600AD47AF4612050C8050854838AB47AD46E6
:100E4600AF3E12054380427F001204A17F40120488
:100E5600A1803675F005E54DA42476F97700802942
:100E6600AD46AF3E12057E8020AF3E12069B80192E
:100E7600AF3E1207268012854B29854A28853E27D4
:100E86007B437D497F4912023AE5402404F582E519
:100E96003F3401F583E06043854082853F83E0FA75
:100EA600E5402401F582E4353FF583E0C39AF54336
:100EB60024FC50277D03AF40AE3F1201E5FB7A00CC
:100EC600EB2404FBE43AFAAD437C00D3EB9DEA9CA9
:100ED60030D202B2E730E7030209ABE5422404F55B
:100EE60082E5413401F583E06003020F607420451A
:100EF6003EFF120139FA4549F54954C0605CE542A6
:100F06002404F582E5413401F583E54CF0E54E70A5
:100F1600467425453EFF120139F543AA4C1A5AF587
:100F260043FAE5422404F582E5413401F583EAF00B
:100F3600700FE5422404F582E5413401F583E54C62
:100F4600F0748055496010E5422404F582E5413489
:100F560001F583E04480F053493FE5422404F582DD
:100F6600E5413401F583E07003021200E5422404F2
:100F7600F582E5413401F583E0B4FF6D7D40AF3E77
:100F86001202B8AF42AE411201FDF5298549288506
:100F96003E277B627D617F5212023A754303E53E2E
:100FA600B48003754307AD4DAF42AE41120211AD99
:100FB60043AF42AE41120211E5422406F582E541F5
:100FC6003401F583E0FD04F0AF42AE411202117D1B
:100FD60000AF42AE41120211E5422404F582E5411A
:100FE6003401F583E4F0021200E5422404F582E5BB
:100FF600413401F583E0547FF545E5422401F5824D
:10100600E43541F583E0854282854183FAE0C39A5F
:1010160014FB7A00AD457C00ED2408FDE43CFCD3CE
:10102600ED9BEC9A30D202B2E720E703021200E50C
:1010360045700302119BE5422404F582E541340123
:10104600F583E054806016E54524DF40108545446D
:10105600754301E53EB48013754305800E75442043
:10106600754300E53EB48003754304E5422401F56B
:1010760082E43541F583E0FA04F0E5422402FDE41A
:101086003541FCED2AF582E43CF583E54DF0E54279
:101096002401F582E43541F583E0FA04F0E54224C3
:1010A60002FDE43541FCED2AF582E43CF583E54397
:1010B600F0E5422406F582E5413401F583E0FA04C1
:1010C600F0E5422401F582E43541F583E0FB04F0C6
:1010D600E5422402FDE43541FCED2BF582E43CF5C6
:1010E60083EAF0E5422401F582E43541F583E0FA2E
:1010F60004F0E5422402FDE43541FCED2AF582E4E4
:101106003CF583E544F0E5422401F582E43541F5FA
:1011160083E0F550E5422402F555E43541F554AF38
:101126003E120139FAE5552550F582E43554F5832A
:10113600EAF00550E545C39544F545E5422404F536
:1011460082E5413401F583E0C39544F01544E54456
:10115600602E907FE3741BF0907FE4743EF0907FE6
:10116600E5E543F0901B3EE0F543E5552550F58255
:10117600E43554F583E543F005501544E54470D253
:10118600E5422401F582E43541F583E550F0E54575
:10119600600302103CE54E703B7427453EFF12018A
:1011A60039F54354F0FA64A0602AAF42AE41120109
:1011B600FDF528854329853E277B427D417F5212D6
:1011C600023AE5422404F582E5413401F58374FFD1
:1011D600F0020EE17D80AF3E1202B8E5422404F52E
:1011E60082E5413401F583E4F07480653E600B745A
:1011F60021453EFF120139020EE1E5422405F58242
:10120600E5413401F583E549F022538EF8438E011A
:10121600907F9C7430F0907F93F0907FE274D2F0D0
:10122600907F957404F0907F9E74FBF0907F987485
:10123600B8F0907F98E054BFF0907F98E04408F0B3
:10124600907F98E054DFF07FBC7E02120036907FDC
:1012560098E054F7F07F2C7E011200367524007D4D
:101266000A7F851200237D0F7F76120023227D00E0
:101276007F0012010C907F98E054F7F0907F98E081
:1012860054DFF0907F9CE4F0907F93F0907F98E09D
:1012960054EFF0907F98E04440F0228C568D578AA8
:1012A600588B59855782855683E054026003021392
:1012B60028E5572401F582E43556F583E0F9EF2455
:1012C60001F582E43EF583E0FA8F828E83FBE0C36C
:1012D6009B14FBE9D39B504AAC02EF2402F55BE476
:1012E6003EF55AAD01E96021855982855883E0FAB9
:1012F600E55B2CF582E4355AF583EAF00559E559A4
:10130600700205580C1DED70DFEF2401F582E43EF6
:10131600F583ECF0E5572401F582E43556F5837440
:1013260040F0228E5C8F5D8C5E8D5F8A608B61855E
:101336005F82855E83E0540260030213C6855D8288
:10134600855C83E0FAE55D2401F582E4355CF5838E
:10135600E0C39AF56224FC50677D03AF5DAE5C1274
:1013660001E52404F563D395625055855D82855C5D
:1013760083E0F564E55D2402F566E4355CF5658594
:101386006362E5636023E5662564F582E43565F509
:1013960083E0856182856083F00561E56170020501
:1013A6006005641562E56270DD855D82855C83E5B6
:1013B60064F0E55F2401F582E4355EF583E563F0CC
:1013C60022907FA17401F0907FD67406F075890192
:1013D60075881043D8201202E51212101203AF7F4F
:1013E6000012047A7F001204A17F401204A1752422
:1013F600017F001201677529007528007527007B9B
:101406006B7D687F6312023A7FC21201394420F570
:101416002775292F7528007B727D657F7612023A23
:10142600757200858C700526756D047989E7B40799
:1014360003756D067977E77005797CE76003436D80
:1014460001AF6D120167907FABE054106009907F89
:10145600AB7410F00213C7907FABE0540860149091
:101466007FAB7408F07F0012016712127443870184
:101476000213C7907FABE054017003021826757102
:101486000075680074086568700302153F75F009F9
:10149600E571A42568901A3B93249B601A24FD608D
:1014A6005D24FC603B24FE602624FB607424FB70F4
:1014B600030217DB0217BD74E82568F582E4347F62
:1014C600F583E0F567547870030217DB0217F174B1
:1014D600E82568F582E4347FF583E0F56B0217DBD7
:1014E60074E82568F582E4347FF583E0FB7A00E44E
:1014F600FDE56EFC4AF56EEB4DF56F0217DB74E801
:101506002568F582E4347FF583E0FF7E007D0812CE
:101516001914E56FFBE4FA4EF56EEF4BF56F021703
:10152600DB74E82568F582E4347FF583E0F56C2406
:10153600F840030217DB0217F175F009E571A425DF
:1015460068901A3B93F575901AB075F00E1218DA7A
:101556000217F17480556760197407556725E0FA1C
:1015660024B4F582E4347FF583E0907F005401F0E3
:1015760080177407556725E0FA24C4F582E4347FA2
:10158600F583E0907F005401F0907F01E4F0907FB6
:10159600B57402F002181A907F00E4F0907F01F013
:1015A600907FB57402F002181A747F5567700302B3
:1015B60017F174805567601F7407556725E0FA2494
:1015C600B4F582E4347FF5837401F07407556790AF
:1015D6007FD74410F0801B7407556725E0FA24C4B2
:1015E600F582E4347FF5837401F0907FD7E5675484
:1015F60007F0907FD7E04420F0907FD7E054DFF0EB
:1016060002181A747F556770030217F174805567C4
:1016160060157407556725E0FA24B4F582E4347F33
:10162600F583E4F002181A7407556725E0FA24C416
:10163600F582E4347FF583E4F002181A75691975AA
:101646006A45907FD4E569F0907FD5E56AF0021887
:101656001A756919756A57907FD4E569F0907FD538
:10166600E56AF002181AE56C25E02408F98769098D
:10167600876AE56CB403607FFF7E0F1200D7FB7AA2
:1016860000C002C0037FFE7E0F1200D7FF7E007DE2
:1016960008121914D0E02FFFD0E03EFEEF2400F52B
:1016A6006AEE3401F569757300AB737A00E56A2B4F
:1016B600FFE5693AFE1200D7FA74002573F582E455
:1016C600347FF583EAF00573E57324EA50DB907FF7
:1016D600B57416F002181A757400E56C25E0240836
:1016E600F987020987038B828A83E06039AB6AAA8D
:1016F60069056ABBFF0205698B828A83E493FA74E3
:10170600002574F582E4347FF583EAF00574E56C10
:1017160025E02408F987020987038B828A83E0FA89
:10172600E574C39A40C7E56C25E02408F9870209E9
:1017360087038B828A83E0907FB5F002181A907F28
:1017460000E519F0907FB57401F002181AE56B6098
:1017560008B4010280030217F1856B1902181A906A
:101766007F00E51AF0907FB57401F002181AE56B58
:101776006008B4010280030217F1856B1A02181A79
:101786007FFF120167AD6BAF6FAE6E1200A37F00D5
:10179600120167AF6FAE6E1200D7FA656B70030267
:1017A600181A8047AF6FAE6E1200D7907F00F09088
:1017B6007FB57401F0805D75F009E571A425689028
:1017C6001A3B93FA74E82568F582E4347FF583E0E2
:1017D600FBEAB5030B0568E56824F7400302148AA3
:1017E6000571E57124F34003021487907FB47403F6
:1017F600F08575297528007527007B437D497F553F
:1018060012023A8015907F00E4F0907F01F0907FFD
:10181600B57402F0907FB47402F0907FAB7401F05F
:101826007B407A7E7DC67C7F7F207E201212A17B44
:10183600277A217D207C207F001208697B807A7EB2
:101846007DB67C7F7F277E211213297BC07A7D7D22
:10185600C87C7F7F2E7E221212A17B357A237D2EB5
:101866007C227F401208697B007A7E7DB87C7F7F70
:10187600357E231213297B407A7D7DCA7C7F7F3C8F
:101886007E241212A17B437A257D3C7C247F801224
:1018960008697B807A7D7DBA7C7F7F437E25121323
:1018A60029C3E58C9570F570E572D39570501E7559
:1018B60029007528008570728570277B747D3E7FB0
:1018C6003E12023AE57224D05003757200858C7080
:0418D60002142C22AA
:1018DA00CAC0E0E4936AA36009A3A3D5F0F5D0E0F7
:1018EA00FA22E493FAA3E493F5828A83D0E0FAD049
:0518FA00E0D0E0E47302
:1018FF00C0F0ED8FF0A4CFC5F0CCA42CCE8DF0A40A
:05190F002EFED0F022C5
:10191400ED540F600AFDC3EF33FFEE33FEDDF72213
:0E192400E493F608A3EFB582F7EEB583F32245
:00000001FF
